:030000000219FDE5
:03000B000200AA46
:03002B000201636C
:03005B000202F5A9
:030073000202E2A4
:1000800002030406080C10182030406080040608A3
:100090000C10182030406080A0C00003070F1F0D17
:1000A0000D0403060D0503030202C2AFC0D0C0E079
:1000B000206214E5256009E473E525F4F58AD2622F
:1000C000D0E0D0D0D2AF3285268AC262E526F46075
:1000D0003630682C20720DD0E0D0D0C282C286C2E9
:1000E00087D2AF32C282C286C287206F13206510CA
:1000F000740AD5E0FDE57BB4010442902100428002
:10010000D0E0D0D0D2AF32758A00C28DD262210049
:1001100001B9306805206502D28201B93068052036
:100120006502D28601B9306805206502D28701B91F
:10013000C28130680A2065077406D5E0FDD28201CD
:10014000B9C28330680A2065077406D5E0FDD286FF
:1001500001B9C29030680A2065077406D5E0FDD267
:100160008701B9C2AFC2AD53E6EFC0D0C0E0D2D371
:10017000D2AFC2CEE52A600720744F152A21CA7873
:1001800000790020742EE580307E01F430E502789D
:10019000FF53DACF207E0343DA20307E0343DA10A8
:1001A000C2D8C271E580307E01F430E50279FFC328
:1001B000E89970CB306103752A40207403752A409A
:1001C000885CD270E86003755F0020740DE52B60D9
:1001D00004152B21DA43DA01C2D820700221EDA8E0
:1001E0005C206102C27020740221EB88227882B602
:1001F000040385222420CF0AD0E0D0D043E610D2D9
:10020000AD32C2CF053A7802E52A60053074021596
:100210002AC3E55C94014005755F00412E756000BE
:10022000756900E55F2401F55F5003755FFF798212
:10023000B7020D306E1DC3E52294324016854C2264
:100240007982B7030E306E0BC3E5229432400479F5
:100250008E8722C3E523952260084004152341625E
:100260000523D8CA0569E56970021569D56A6975FB
:100270006A017808E56B60497805C3E569956B40CC
:1002800057C3E569956C50087801756A0302029CB2
:10029000C3E569956D50057801756A01C3E56295FE
:1002A00024401E7982B7040241CD206E1485246259
:1002B000E569046003856B69756A0175233C020278
:1002C000D8E5622850057562FF41CDF562E562040C
:1002D00070067560FF7569FFD0E0D0D043E610D29C
:1002E000AD32C2AF53E67F7592FA7593FFC2607567
:1002F0009104D2AF32C2AF53E6EFC2ADC0D0C0E07E
:10030000C0F0D2D3D2AFA8FBA9FCC2D83071026131
:100310005C53DACF207E0343DA10307E0343DA20C9
:10032000D271E580307E01F420E5026133882789AF
:1003300028A14153DACF207E0343DA20307E0343E5
:10034000DA10C2D8C271307402A12D7800E5803075
:100350007E01F430E502A12D885CA11553DACF208F
:100360007E0343DA20307E0343DA10C2712061023B
:10037000813553DACF207E0343DA10307E0343DA2F
:1003800020C2D8D27188578958C3E89555F8E995A5
:1003900056F97B007E087A00C3E8948CE9940050FB
:1003A00005755B008127882178A2E6A8216055C3E6
:1003B000E894C8E994005008E4D2E4FB7A0A810288
:1003C000C3E89468E994015008E4D2E3FB7A0F8112
:1003D00002C3E894D0E994025008E4D2E2FB7A1E0A
:1003E0008102C3E894A0E994055008E4D2E1FB7AC5
:1003F0003C8102C3E89498E994085008E4D2E0FBF9
:100400007A787E00C3E89559FCE9955AFD30E70AF1
:10041000ECF42401FCEDF43400FD755B00C3EC9AB0
:10042000ED9E5003755B018859895A85575585584B
:10043000567802A115C3E89527F8E99528F9307C8C
:100440000281F9307B0281F9307A0281F220750253
:100450008158E9FDE8FC8177E9C313F9E813F83026
:10046000790281F2E9C313F9E813F830780281F2D6
:0F047000E9C313FDE813FC20612CC3EC941CEDD1
:10047F0094024002818EED701EC3EC94C850180593
:10048F0029E52970021529C3E529940A5002A12DE7
:10049F00755C00D270A12DE529600215297400202A
:1004AF007F037896E624FAFEE43400FFC3EC9EFC4B
:1004BF00ED9FFD50067800790081F9C3EC94FFEDB4
:1004CF009400400678FF790081F9EC8572F0A4C59D
:1004DF00F0A2F733F87900400302051578FF790091
:1004EF00020515E9C313F9E813F8307C0EE9600231
:1004FF0078FFC3E81338F8E43400F9C3E894FFE950
:10050F009400400278FF885CD270206102A12D74A4
:10051F001FF4552F4BF52FC274EB7002D274752A4E
:10052F0040307403752A0A306102A14120740353CD
:10053F00DAFE207403752B20D0F0D0E0D0D0D2ADEE
:10054F0043E6103279010205717903020571790AC8
:10055F00020571791E020571796402057179C8026D
:10056F0005717817E4D5E0FDD8FAD9F6227A147B15
:10057F00780205987A107B8C0205987A0D7BB4026D
:10058F0005987A0B7BC8020598E573D5E0012279AF
:10059F0002E4C283D5E0FDD286D5E0FDC286D5E068
:1005AF00FDD283D5E0FDE920E002D28230E002D215
:1005BF0087E573D5E0FDE920E002C28230E002C298
:1005CF00877496D5E0FDD9C9EAF8D5E0FDD8FBDBF5
:1005DF00B8C28322C37C007D0075F00005F0EA33BA
:1005EF00FAEB33FB50F6EB13FBEA13FAC3E9FFE820
:1005FF00FEE89AF8E99BF95004EFF9EEF8B3EC3303
:10060F00FCED33FDD5F0DFEDF9ECF822E889F08A47
:10061F0020D2D4F8A9F07B0030F70B7BFFF4240134
:10062F00F8E9F43400F9E88520F0A4ADF0F8E98595
:10063F0020F0A4AFF0FEED2EF974003FFA7C04C356
:10064F00EA13FAE913F9E813F8DCF48BF030F70A40
:10065F00E8F42401F8E9F43400F9E889F0C2D4F899
:10066F00A9F0227882B60403020711C3E55C94193E
:10067F00401EE52D54067018206E3678057994E7E4
:10068F00146007780A1460027812C3E54198401F7E
:10069F00306E098564627569FF756A01852224E4ED
:1006AF00F544F545F546F547F548C26E020711D2F8
:1006BF006E7994E7147013E523F43333F913F8E9E3
:1006CF00540104F9E854FE020705E714147014E509
:1006DF0023F4333333F913F8E9540304F9E854FCE2
:1006EF0002070DE523F433333333F913F8E95407D5
:1006FF000404F9E854F8C39440F8E99400F98844E5
:10070F00894522C3E54113F9E54013F8C3E5449841
:10071F00F8E54599F9500CC3E89480E994FF401629
:10072F00020749C3E8947FE9940050030207497810
:10073F007F7900020749788079FF8849894A22E545
:10074F00492546F8E54A3547F9854A20E43007013F
:10075F00F43548FA30E709C3EA94F04015020787E9
:10076F00C3EA940F500302078778FF79FF7A0F02CD
:10077F000787780079007AF0C3E5249561500AC3A2
:10078F0074019524500B0207A5E54A20E70E0207D6
:10079F00A5E54A30E706884689478A482278A5E6C4
:1007AF00FAC3E54933F8E54A33F9D11BE930E70BD2
:1007BF00C3E89480E994FF4013E1DFC3E8947FE935
:1007CF0094005002E1DF787F7900E1DF788079FFD4
:1007DF00E820E715C3E52398F84009C3E8940140E2
:1007EF00030208067801020806E8F424012523F81D
:1007FF00400302080678FF884B2278A6E6FAA8473E
:10080F00A94812061BE930E70CC3E89401E994FFED
:10081F00401602083BC3E894FFE994005003020816
:10082F003B78FF790002083B780179FFE920E71553
:10083F00C3E54B98F84009C3E894014003020862EE
:10084F007801020862E8F42401254BF840030208FE
:10085F006278FF88242278FF20692879A1E7602336
:0D086F00E541601F74FF8541F0848539F07C
:10087C00306A0375F005A4F8C5F0600278FFC3E890
:10088C0095645002A864886322C3E5409440E54116
:10089C009401E56350031401A6046002F563227809
:1008AC0083E6F520120F2875E89012055375E89031
:1008BC0030EDFDA8BDA9BE120FCF756E00756F008F
:1008CC00C3740013FD7400606613FC74002CFC747C
:1008DC00003DFDECFAEDFBC3E89AE99B4014E56E94
:1008EC002400F56EE56F3400F56FEA2CFAEB3DFB56
:1008FC0080E5AE6EAF6FC3E56F13F9E56E13F8C309
:10090C00E913F9E813F87A03C3E913F9E813F8DAF1
:10091C00F7AA201A7009756E00756F0002093B1A50
:10092C00EA6008EE28FEEF39FFDAF88E6E8F6F2240
:10093C0075E890227883E6FF30EDF9A8BDA9BE05D5
:10094C0070C3E57094084052757000E9FA79A0E71D
:10095C006044EA7007E571601B020974C3E8957185
:10096C006010E5715006600C140209800460F902F5
:10097C000980E571F571C39467401B7561C0C39420
:10098C00044013756180C39404400B756140C3949B
:10099C0004400375610075BB0B22EFC39401601F0B
:1009AC007400601BC3E894FFE994035012C3E895EC
:1009BC006EE9956F5009E561600C15610209D2E58D
:1009CC0061F460020561A861C3E524985002A82473
:1009DC00C3E89562400AA862E562F460038562612F
:1009EC0088258826E570B4070375BB10227432790C
:1009FC00A787F0A4C5F0A2F733F8C3E895614002CD
:100A0C00A86188228824882588268864227540005D
:100A1C007541F022C2AF75C820A8CCA9CDAA3A3036
:100A2C00CF010A75C824D2AFAB3BAC3C883B893CA8
:100A3C00C3E89BF8E99C206908F9306602613141F2
:100A4C008BAD3D8A3DF9EA9DFA600678FF79FF414E
:100A5C0070AE3EAF3F8B3E8C3FA83BA93CC3E89E9B
:100A6C00F8E99FF9C3E54113FBE54013FAE82AF5D1
:100A7C0040E93BF54150067540FF7541FF41D8AA4E
:100A8C0040AB41AC40AD417E047F02C3EB940440CB
:100A9C000D1E1FC3EB94084005206A021E1FC3EDF8
:100AAC0013FDEC13FCDEF7C3EA9CFAEB9DFBEF6045
:100ABC0009C3E913F9E813F8DFF7EA28FAEB39FB75
:100ACC008A408B4150067BFF8B408B41C3EB9402D9
:100ADC005002D2663069047F0361037892E6FFC34B
:100AEC00E537948240110FC3E53794A040010FC342
:100AFC00EF940640027F057E02E541C4540FF9E5F0
:100B0C0041C454F0F8E540C4540F28F8C3E89EFAE9
:100B1C00E99400FB4009C3EA9402EB940050047A78
:100B2C0002E4FB617DAA40AB41EBC4FEEAC4540F66
:100B3C004EFCC3EA9CFAEB9400FBC3E813C313F816
:100B4C00EA28FAEB3400FB8A408B41C3EB94024059
:100B5C0002C2667802EBC4FE7B00EAC4540F4EFA64
:100B6C00C3EA98FA4005C3940250027A027892E6DE
:100B7C00FF306002617D855192855293D26043E6CD
:100B8C0080C3E49AF8E49BF93066028109E8FAE93B
:100B9C00FBD3E913FDE813FC88518952C3EF94038E
:100BAC006038EF20E00DE82CF8E93DF9ECFAEDFBAC
:100BBC00020BD2E828F8E939F9C3E82402F8E93441
:100BCC0000F97AFE7BFFC3EF9403400E8A538B54DB
:100BDC00884D894E8C4F8D50813D885389548A4D58
:100BEC008B4E8C4F8D503069127553F07554FF75C8
:100BFC004FF07550FF7551F07552FF813DE8FAD3F7
:100C0C00E813FC8851C3EF94036020EF20E007E861
:100C1C002CF8ECFA8129E8282402F87AFEC3EF9428
:100C2C000340088A53884D8C4F813D88538A4D8CE4
:100C3C004FE568C3335002646BF56830600281473E
:100C4C00753402D26043E680E52D54066034A8402A
:100C5C00A941C3E913F9E813F8C3E913F9E813F848
:0F0C6C00306904E92440F9C2AF53E67F75910067
:100C7B00C3E498F594E499F595759104D26043E635
:100C8B0080D2AF22D264754300752000306C03759F
:100C9B002040020CAED264754300752040306C03CB
:100CAB0075200078017901206620E52D540660023D
:100CBB00C2647914E541C313700104F8C394144062
:100CCB00027814306904781B791B206010E54360AF
:100CDB000C306903D53404D26DA158914F0543E50F
:100CEB00BF5440B52002A14230690908C3E89940BE
:100CFB00011881D520640A08C3E899400281AE81AE
:100D0B00D5C264C2AF53E67F7591003066127594FD
:100D1B00007595F8759104D26043E680D2AF81AE31
:100D2B00E5417EFFC3334005C3334001FEC3E49E60
:100D3B00759400F595A11FC3E5339401500281AE64
:100D4B0030640281AED802A15681D5C26DC2AF53B9
:100D5B00E67F759100855394855495759104854D67
:100D6B0092854E93D26043E680D2AFE52D54066058
:100D7B0008206A020533020D94306D0D206C0A2099
:100D8B0064071581158102164922780030640278B8
:100D9B0001E53775F007A4F9E5F028F5F0E9A2F0C5
:100DAB0013A2F113A2F213F537C3947850037537DE
:100DBB0078C3E53795384008D265C282C286C287B0
:100DCB00306002A1CB854F92855093D26043E68071
:100DDB0022207D16C2AF754202C283D281306202DD
:100DEB00D287D2AF75AA23020FCCC2AF754202C213
:100DFB0083D290306202D282D2AF75AA23020FCC7B
:100E0B00307243207D20C2AF754203900141757B48
:100E1B0008C287C290306204D286C129D283D2AF76
:100E2B0075AA24020FCCC2AF754203900141757BAA
:100E3B0008C282C281306204D286C149D283D2AF4A
:100E4B0075AA21020FCC207D17C2AF75420390010A
:100E5B001CC287306202D286D2AF75AA24020FCC95
:100E6B00C2AF75420390011CC282306202D286D29D
:100E7B00AF75AA21020FCC207D16C2AF754204C2FA
:100E8B0081D290306202D286D2AF75AA21020FCCEA
:100E9B00C2AF754204C290D281306202D286D2AF09
:100EAB0075AA24020FCC307243207D20C2AF75424D
:100EBB0005900130757B02C286C283306204D282F8
:100ECB00C1CFD281D2AF75AA23020FCCC2AF75426C
:100EDB0005900152757B01C286C283306204D287B2
:100EEB00C1EFD290D2AF75AA23020FCC207D17C2CF
:100EFB00AF754205900112C286306202D282D2AF28
:100F0B0075AA23020FCCC2AF754205900126C2868B
:100F1B003062EBD287D2AF75AA23020FCC207D169D
:100F2B00C2AF754206C290D283306202D282D2AF78
:100F3B0075AA24020FCCC2AF754206C281D2833090
:100F4B006202D287D2AF75AA21020FCC3072442035
:100F5B007D20C2AF754201900152757B01C282C2E6
:100F6B0081306204D287E175D290D2AF75AA21028B
:100F7B000FCCC2AF754201900130757B02C287C2A4
:100F8B0090306205D282020F96D281D2AF75AA241D
:100F9B00020FCC207D17C2AF754201900126C28291
:100FAB00306202D287D2AF75AA21020FCCC2AF75C5
:100FBB004201900112C287306202D282D2AF75AA6F
:100FCB0024C26522900110757B00C282C286C28743
:100FDB00C281C283C290C2622278807607087607EC
:100FEB000876010876040876FF0876FF08760A086B
:100FFB007602087601087601788C7601087600086F
:10100B0076B40876FF0876FF0876FF087603087635
:10101B00FF0876010876FF0876250876D0087678E3
:10102B000876C80876040876FF087601087600086B
:10103B00767A08760A087601087601087600087633
:10104B00FF087600227887E6FFC272BF0302D272D6
:10105B007888C27DE630E102D27DC27E7889E630A7
:0F106B00E102D27EC3EF94026008758E01D2734A
:10107A00021082758E00C273227880E61490008076
:10108A009378A5F67881E6149000809378A6F6788E
:10109A0086E61490008D9378A7F6789FE6F8700597
:1010AA00756B0001C9C3E8941140027811E8282839
:1010BA00F56B256B256B28F56C256B2828F56D7863
:1010CA0086E6F539C394025003753902789CE675B1
:1010DA0038FFB402037538A0B4030375388278A3C5
:1010EA00E61490009A93F566120FCF22227896E6BC
:1010FA00FA7897E6FB7888E6B40305C3EB940EFB0F
:10110A00307F047A007BFFC3EB9AFCC394825002BF
:10111A007C827572000572EC8572F0A4C3E5F094C6
:10112A007D40F222D27F11F71205621205627A001F
:10113A007B007C10120558E55C2AFA74003BFBDC44
:10114A00F37C04C3EB13FBEA13FADCF7FEC27F114C
:10115A00F722757C00757D00E5EF20E60375200017
:10116A000520903FFFE520146006901FFF146000E1
:10117A009304600375EF167597DE7597AD7581C098
:10118A0043FF8012055375EF0675A900E5C72402CF
:10119A0020E70DF521E5B120E0068521C743B1011D
:1011AA00120FCF75803175A4CE75F1FF75D4DF7536
:1011BA0090FE75A50175F2E175D50075A60175E376
:1011CA004075E201120FCFE4F8F6D8FD75680112F6
:1011DA000FE41216A078988673753001C2AF120513
:1011EA006C12057C12056212058312056212058AC9
:1011FA001205621217D312056C12056C120567C22A
:10120A00AF757C00757D0078FA79FA308507D9FBCD
:10121A00D8F7021C001150118311F611F77898863D
:10122A0073120FCF75881075890275C824759104D9
:10123A0075D84075A82275B80275E690759B8075B9
:10124A009D0075BF8075AB0075D10C75BC5975BB17
:10125A000B75E88075B201120553D2AF1208AB754F
:10126A00360053DACF207E0343DA20307E0343DA96
:10127A001043DA01C2D8C27112056CD2617B037ABB
:10128A000CE55B70077A0CDB030212091205622077
:10129A007003021209C270E55CC3940240E1E52FB3
:1012AA00541F855E5DF55EB55DD5DAD5C26153DA48
:1012BA00CF207E0343DA20307E0343DA10C2D8C23D
:1012CA007178A2E67008D274E52F54E0F52FC27542
:1012DA00752900120567307409C3E529940A40028A
:1012EA00D27512055878023074027800C3E55C980A
:1012FA0040F0C2AF12057C12057C12057CD2AF12F7
:10130A00056C754C00120558788CE6C3940150039D
:10131A000213FCE530C3940150030213FC757CA54B
:10132A00757DF1207435C3E55C94FF50030213FC0C
:10133A00C2AF120591D2AF120567C3E55C940150A2
:10134A00EFC2AF12057C12055D12057CD2AF120501
:10135A0067C3E55C94FF40E90218587F05D27F1104
:10136A00F7120567C2AFC27F11F7AE5CC3E55C94A2
:10137A007FD2AF5002810C120553C2AF120591D22F
:10138A00AFDFDA312EC3EE94057897F612056C12A8
:10139A0017DB7F0AD27F11F7120567C2AFC27F112E
:1013AA00F7AE5CC3E55C947FD2AF50E6120553C238
:1013BA00AF12057C12055D12057CD2AFDFD6312E45
:1013CA00EE24037896F6F87997E7C3948240039857
:1013DA005006E824827897F612056C1216EE121857
:1013EA000A12056711F7C3E55C94FF5002612702F0
:1013FA001858757C00757D00C3E55C954C400385E3
:10140A005C4C12056778017988E7B403027805C352
:10141A00E55C984002610FC2AF1205911205911264
:10142A000591D2AF12056C753000E4F531F532053D
:10143A0031E531F4703F0532789AE6781914601272
:10144A00783214600D787D14600878FA1460037598
:10145A003200C3E53298401D120FCF1205531532E0
:0E146A0075310078998673C2AF120591D2AF2A
:101478007898867312056712055DE52A7005307441
:1014880002410978012074027806C3E55C9840A1FE
:10149800120567E52A7003021209C2AF120FCFE4E2
:1014A800F522F523F524F525F526F567D2AF7885DD
:1014B800E6C333F565E4F544F545F546F547F548E3
:1014C800F570F52CF52DF53775700875BB101205FC
:1014D8005312093C30EDFDA8BDA9BEE97001F8889A
:1014E8007112094075700875BB101150C2AF756153
:1014F800FF1209F9852261852262852263D2AF75C0
:101508002201752401752501752601856069756AB2
:10151800017888E6B40307C27D307602D27DD268AE
:10152800D269753300120F28120F57120A19120ABE
:1015380020120A19120A20120A19120CA012067295
:10154800120D95120DDC120A20120C8F306E031248
:101558000712206603120865306603120895120DFB
:1015680095120E0B120A20120CA0306E0312074EB1
:10157800120D95120E82120A20120C8F306E031271
:1015880007AC120D95120EB1120A20120CA0306E83
:1015980003120809120D95120F28120A2012093C8D
:1015A800120C8F120D95120F57120940120A203093
:1015B800692C856461856462856069756A0179183A
:1015C8007A0CC3E533994009C269D26A8A35021593
:1015D800E6C3E55C94014003021542021651306AE5
:1015E80025206C22E535147006C26AD26BA142F53B
:1015F80035C3E55C940140030215427888E6C3943C
:10160800036003021651753600C3E55F9401400973
:10161800856462856069756A0178FA79A4E7600271
:101628007803C3E55F985021307404E52A601A787E
:10163800F0306C058564617820C3E541985002A1BB
:10164800420536E55C6002C154753600C2AF120F20
:10165800CF7887E6FE760211507887EEF6E4F52219
:10166800F523F524F525F526F565752C00752D006F
:10167800D2AF120567120FCF78A4E66006D282D2E5
:1016880086D287307406E52A70024109788DE6C350
:101698009401400241EC8134901A0D7820121730E1
:1016A800E520B4A50CA3121730E520B45A0302169E
:1016B800CE757CA5757DF1120FE41216EE757C00CF
:1016C800757D000216ED901A0378807B0A12173098
:1016D800A308DBF9901A0F788C7B19121730A3082E
:1016E800DBF9901A2822C2AF121773121750901AFA
:1016F80000740E121735A37409121735A374151246
:101708001735901A0378807B0A121734A308DBF97F
:10171800901A0F788C7B19121734A308DBF912176B
:1017280086121764901A2822E493F622E6438F0162
:10173800538FFDFFC3E583941C400122EF857CB7DE
:10174800857DB7F0538FFE22438F02438F01857C3E
:10175800B7857DB7901A0DF0538FFC22901A0D743F
:10176800A5F135901A0E745AF135227A3079D0786D
:1017780020901A40F130E520F709A3DAF7227A30F1
:1017880079D0901A40E7F13509A3DAF922AB74A8A9
:1017980075BB01027980BB02027981BB03027982A1
:1017A800BB04027994BB05027983BB06027986BB28
:1017B80007027992BB08027987BB0902799CBB0AA8
:1017C800027988BB0B027989E8F7227C0512056C3F
:1017D800DCFB22C2AF12057C12058312058A1205B2
:1017E8009112055D12057C12058312058A12059176
:1017F80012055D12057C12058312058A120591D225
:10180800AF22C2AF12059112058A12058312057C18
:1018180012055D12059112058A12058312057C12C4
:10182800055D12059112058A12058312057CD2AF57
:1018380022AE74AF75C2AF12057C12057C12057C0E
:1018480012055DDEF212059112055DDFF8D2AF22B6
:101858001217DB1217D31217D3757401757501753A
:0F186800760011397C05AD5C12056CC3ED955C03
:1018770070F5C3E55C9401400AC3E55C94FF40370B
:1018870002189B1217951216EE1217DBC2AF75EFEF
:10189700161217D3DCD10576C3E576940350028080
:1018A700C21217D30575E5741490009F93F808C307
:1018B700E57598500280A91217D31217D30574C380
:1018C700E574940C50028095120FE41216EEC2AF25
:0618D70075EF161217D395
:0319FD0002115C78
:101A00000E091507070104FFFF0A020101A55A018B
:101A100000B4FFFFFF03FF01FF25D078C804FF01DA
:091A200000FF0A010100FF00FFB4
:101A4000234D5232355F3135412320202020202084
:101A500023424C48454C492346383530232020202A
:101A60002020202020202020202020202020202076
:101C0000C2AFC2D37597DE7597AD7581C075A90057
:101C100043FF80752438752503B1DB7529A5752A26
:101C2000F175E34043F12053A4DF75D4FFD2857DE5
:101C3000FA780379E67C10752200752300901DE880
:101C40007B0675249875250130850281482085081A
:101C5000D8FBD9F9DCF781BA308508D8FBD9F9DC93
:101C6000F781BAB19BE493A3C39A6004DDC381BA40
:101C7000DBDBB18D600281317B08E493FAA3B16EA6
:101C8000DBF87A30B16E752200752300B18DEAFC65
:101C9000EBFDC3ED94FE400EB18D8A278B28ED300D
:101CA000E0048A828B83B18D7AC270D8C3ED94FE32
:101CB000601950CEBD0029EC600F7520007521FF22
:101CC000752900752A000200008100A827A92808AC
:101CD00009D804D90281DDB191EAF281D10D81A642
:101CE000C3ED94035051EDA2E092007AC5C3E582A2
:101CF0009400E583941C508C200010438F02438F86
:101D0000018529B7852AB7F0300027A827A9280818
:101D100009438F01538FFDD804D902A132C3E58353
:101D2000941C4003A3A117E28529B7852AB7F0A325
:101D3000A117538FFC81827AC1BD030CE493A3FAEF
:101D4000B152DCF8B14A81828184AA22AB23B16E00
:101D5000EBFAEA6222752608C3E52313F523E52290
:101D600013F52250066323A0632201D526EAB1DBD6
:101D7000B1DB75260AEAF4200102D285300102C2E5
:101D800085B1DBC3134002C201D526EB22B191EA33
:101D9000FB208502A191308502A196752608AE240C
:101DA000AF25C3EF13FFEE13FEB1DFB1DBC3EA13C0
:101DB0003085024480FA30E703632201C3E5231330
:101DC000F523E52213F52250066323A0632201D5F3
:101DD00026D9E52265236523F52222AE24AF250E00
:101DE0000FDEFEDFFCD20122424C48656C693437BD
:061DF0003164F850060109
:00000001FF
